:030000000240ECCF
:0C40EC0078FFE4F6D8FD75816F024133C7
:10134D000A53746172743A20004950436F6E6E6592
:10135D0063745245510A004950436F6E6E65637454
:10136D00003E432C562C52432CC0E4E0EFF2E5F046
:10137D0020D1E8EDEAEEEC49500A003E432C4D41F8
:10138D00432C25303262583A25303262583A253096
:10139D003262583A25303262583A25303262583A24
:1013AD0025303262582C4D414320E0E4F0E5F10A3E
:1013BD00003E432C5645522C20332E3120EEF22088
:1013CD0025732025732CC2E5F0F1E8FF204950204C
:1013DD00ECEEE4F3EBFF0A004E6F76203033203253
:1013ED003030370030383A35313A3336003E432C01
:1013FD004C442C50524F473A2020202020202020B2
:10140D0020202020202020202020202020202020CF
:10141D0020202020202020202020202020202020BF
:10142D0020202020202020202020202020202020AF
:10143D00202020202020202020202020202CC4E02F
:10144D00F2E020EFF0EEF8E8E2EAE828F4E0E9EB6C
:10145D00290A003E2A2C312CCEF1EDEEE2EDFBE512
:10146D0020EFE0F0E0ECE5F2F0FB20F1E5F2E5E253
:10147D00EEE3EE20E8EDF2E5F0F4E5E9F1E00A0047
:10148D003E412C4130312C2562752E2562752E255D
:10149D0062752E2562752C495020E0E4F0E5F120AF
:1014AD00E0E4E0EFF2E5F0E00A003E412C4130329D
:1014BD002C2562752E2562752E2562752E25627579
:1014CD002C495020E0E4F0E5F120EEF1ED2E20F175
:1014DD00E5F0E2E5F0E00A003E412C4130332C25E9
:1014ED0062752E2562752E2562752E2562752C4925
:1014FD005020E0E4F0E5F120F0E5E72E20F1E5F0F5
:10150D00E2E5F0E00A003E412C4130342C256275B5
:10151D002E2562752E2562752E2562752CCCE0F177
:10152D00EAE020F1E5F2E80A003E412C4130352C8D
:10153D002562752E2562752E2562752E2562752CF8
:10154D00D8EBFEE70A003E532C4130362C25627550
:10155D002CC2F0E5ECFF20EEE6E8E42E20EAE2E80E
:10156D00F2E0EDF6E8E820282A3130ECF1290A0006
:10157D003E2A2C312CC4EEEF2E20EFE0F0E0ECE50E
:10158D00F2F0FB20F1E5F2E5E2EEE3EE20E8EDF21C
:10159D00E5F0F4E5E9F1E00A003E422C5330312C40
:1015AD002562752CC6E4E0F2FC20E7E0EFF0EEF1E9
:1015BD00E020F1EEE5E4E8EDE5EDE8FF20EEF220C8
:1015CD00F1E5F0E2E5F0E00A003E422C5330322C1A
:1015DD002562752CCEE1ECE5ED20F120F1E5F0E290
:1015ED00E5F0EEEC20E1E5E720EAE2E8F2E0EDF6E9
:1015FD00E8E90A003E422C5330332C2562752CCF7E
:10160D00E5F0E5E7E0EFF3F1EA20EFF0E820EFEEAB
:10161D00F2E5F0E520F1E2FFE7E820F120F1E5F059
:10162D00E2E5F0EEEC0A003E422C5330342C2562FC
:10163D00752CCDE5F220EFE5F0E5E4E0F7E820E4E8
:10164D00E8E0E3EDEEF1F2E8EAE820E220F1E5F082
:10165D00E2E5F00A003E422C5330352C2562752C04
:10166D00CAE0EDE0EB20F8E8F0EEEAEEE2E5F8E0B6
:10167D00F2E5EBFCEDEEE3EE20EEE1ECE5EDE00A5C
:10168D00003E532C5330362C2530326258253032E3
:10169D006258253032625825303262582530326218
:1016AD005825303262582C4D414320E0E4F0E5F1ED
:1016BD0020F8E8F0EEEAEEE2E5F8E0F2E5EBFCED1D
:1016CD00EEE3EE20EEE1ECE5EDE00A003E454E44A2
:1016DD000A0044756D7058202020202030302030B5
:1016ED003120303220303320303420303520303628
:1016FD002030372030382030392030412030422002
:10170D0030432030442030452030460A003A200036
:10171D000A0044756D704420202020203030203088
:10172D0031203032203033203034203035203036E7
:10173D0020303720303820303920304120304220C1
:10174D0030432030442030452030460A0045727227
:10175D00206B657900526420656570726F6D0A00AB
:10176D005264204D454D0A00526420436F64650A52
:10177D000044656275674950204F4E0A004465620A
:10178D0075674950204F46460A0044656275675596
:10179D00736572204F6E0A004465627567557365F7
:1017AD0072204F46460A0044656275674D73672087
:1017BD004F6E0A0044656275674D7367204F46464C
:1017CD000A00436F6E666967206C6F636B210A00B8
:1017DD00577220656570726F6D0A002053617665D2
:1017ED0020656570726F6D210A00457272204D4142
:1017FD004321004C6F61643E3E002A003C41303174
:10180D003D003C4130323D003C4130333D003C41D8
:10181D0030343D003C4130353D003C4130363D00DB
:10182D004E4F4950004C494E4B434F4E545200546D
:10183D0052415353004652004E4F4C494E4B0049B6
:10184D004E49004E4F4449414700003C21003C5356
:10185D0030313D003C5330323D003C5330333D0080
:10186D003C5330343D003C5330353D003C53303615
:10187D003D00FF182DFF1832FF183CFF1842FF18CE
:0A188D0045FF184CFF1850FF1857D4
:064B2C00010B000109006D
:104ABE00C2AFC28E438910758BFF758DB7D2ABD244
:044ACE008ED2AF22B3
:03001B00023DF8AB
:103DF800C0E0C083C082C0D0C2AFC28E758BFF75D1
:103E08008DB720060675A61E75A6E10509D202E53E
:103E18000B6002050BE50AD394014002150A050E52
:103E2800E50E540F7050D20DE50E543F701AD200B3
:103E3800907AF2E0601204F0E0D394B4400A9080E3
:103E4800007480F0C2AF80FE907AEDE0600204F06A
:103E5800907569E0600214F0907AF3E0D394014021
:103E680003E014F0300502050CE50DD3946440041A
:103E7800D2068002050DE508D3940140021508D248
:0C3E88008ED2AFD0D0D082D083D0E032F8
:10087D00C20A7D027C007F07124A708F26E526642E
:10088D006060097D017F601249C3D20AE4FDFC7FDF
:10089D000B124A708F26E52630E6097D04E4FF121F
:1008AD0049E7D20A7D017C007F07124A708F26E549
:1008BD00267008FD7FFF1249C3D20A300A03126069
:1008CD0000C2AFC288C2A8C2AA758900123E94D2D6
:1008DD00AF9077B17403F0A374CCF0E49077B0F0DF
:1008ED00123671EF600312266412245DC2061246A1
:1008FD00909077BDE0C3940350037403F0D20AC205
:10090D000CC20BD293200A077E137F4D123757E48A
:10091D009079DDF0124ABEC2AFA37408F090771C37
:10092D007424F0E4A3F09077A6E090771EF0907712
:10093D00A7E090771FF09077A8E0907720F0907760
:10094D00A9E0907721F09077AAE0907722F0907748
:10095D00ABE0907723F0750A01E49079DFF0C207E0
:10096D00C208D2AF75A70775A61E75A6E112499CE0
:10097D00200A19AF267E007D031239F6E4FF123DE1
:10098D004E7E777FDDE4FB7D01123BA6907AF2E08F
:10099D0060037401F0E4907569F0A37455F0A374CD
:1009AD0081F0E4F50CE4F50D907569E07003121E0D
:1009BD00ED907AF3E0B401119080007410F0E490A2
:1009CD007AF3F0D20AD20BD20C908008E0F52630E3
:1009DD00E405D2077410F0E52630E508D2099080C1
:1009ED00087420F0E52630E608D20890800874409F
:1009FD00F0E50CD394034023908002E4F090800145
:100A0D00F0908000F0E50CD39406400FE4F50CC295
:100A1D00039079DFF0750A011246909080A0E07086
:100A2D00031244819080B8E070031244FB9080D093
:100A3D00E07003124575908000E0701330071012BE
:100A4D00356D907799EFF0D3940040031200269006
:100A5D008002E07006908000E06005D2050209B2C8
:100A6D00C205E4F50C907569E060030209B2300926
:100A7D0012123097907799EFF0D394004005E0FF74
:100A8D00124AE1200803020C0C122F22907799EFE5
:100A9D00F070030209B29077DDE054BF247F70033C
:100AAD00020B6F147003020B4724026003020BA2AA
:100ABD00200A077E137F56123757300E74200371AC
:100ACD009077B5E0FF70069077B9E06055907AE9C0
:100ADD00E0FEB50722A3E0FF9077B6E0B5071890CA
:100AED007AEBE0FF9077B7E0B5070C907AECE0FF7A
:100AFD009077B8E06F602B9077B9E06E7033907A95
:100B0D00EAE0FF9077BAE0B50727907AEBE0FF9027
:100B1D0077BBE0B5071B907AECE0FF9077BCE0B5B2
:100B2D00070F9079DF7401F0120021750A01020C94
:100B3D000C907AE974FFF0020C0C907AF2E06003ED
:100B4D007401F0907AE1E0FF9077DFE06F600302CF
:100B5D000C0C907AE1E004F0E4F50A9079DDF002F6
:100B6D000C0C300303020C0C9077ACE070030209FF
:100B7D00B2124B41D203E4F50A9079DDF0907AED93
:100B8D0004F0E4907AE0F0A3F0200A737E137F6402
:100B9D00123757806A907AF2E060037401F03003E7
:100BAD00529077DDE020E74B9077DFE0FF907AE021
:100BBD00E0FE6F600D907AE8E07007EE146F703F05
:100BCD008013907AE0E004F0907799E0FFD39404DD
:100BDD0040031247779074657482F0A37401F0900E
:100BED0077DFE0907467F07E747F657D03124406B5
:100BFD000209B2300E09200306907AE974FFF02045
:100C0D000303020CC1E50A706B12486AEF60207E87
:100C1D00787FDD9078DEE02404FD124406907AE8BA
:100C2D00E060030209B29077BDE0F50A0209B290C7
:100C3D007AEDE0D3943C403C907AE8E07036907ABF
:100C4D00ED04F090771BE0702B124B22E49078DDD1
:100C5D00F0A37412F0907AE1E09078DFF0A374FDC8
:100C6D00F090756C63A2019078E163A2017F12127E
:100C7D002B09809B124B17EF60159074657483F0F0
:100C8D00E4A3F07E747F657D021244060209B2E58D
:100C9D000A640160030209B29079DDE004F0E0C35B
:100CAD0094055003020C1CC203E49079DFF012008E
:100CBD00210209B2E50A640160030209B29079DFED
:100CCD00E014604024FE603C147003020DA924045E
:100CDD0060030209B2E4F50C200E139079DF740461
:100CED00F09079DDE05401F0750A010209B2E4904B
:100CFD0079DFF09079DD04F0750AC8907AE974FF18
:100D0D00F00209B2907AE9E07003020D989078DD57
:100D1D007480F09078DF7401F0E4A3F0A304F0A3E5
:100D2D007430F0A3747BF0E4F52674E42526F58287
:100D3D00E43478F583747DF074E52526F582E4348A
:100D4D0078F583E4F0E52624079078DEF07C7A7D53
:100D5D00E99077B1E0FAA3E0FB7F021242827E7840
:100D6D007FDDE5262409FD124406907AE8E0601B3C
:100D7D00124B41D203E4F50A9079DDF0907AED043F
:100D8D00F0E4907AE0F0A3F00209B29079DF7404F8
:100D9D00F09077BDE02432F50A0209B2908002741A
:100DAD0010F0750A039079DDE06401FFF09079DFB2
:100DBD007401F0EF70199077B9E06013FCA3E0FDBA
:100DCD00A3E0FEA3E0FF907AE91223130209B2908B
:100DDD0077B5E0FCA3E0FDA3E0FEA3E0FF907AE988
:080DED001223130209B280FE7B
:010DF50022DB
:100026009077DEE0B444047F0180027F009077DDA4
:10003600E0B447047E0180027E00EE5F604A90775E
:10004600A6E09077DFF09077A7E09077E0F09077E2
:10005600A8E09077E1F09077A9E09077E2F09077CA
:10006600AAE09077E3F09077ABE09077E4F09077B2
:10007600DE7452F090771563A2019080A863A20106
:100086007F06122B09020873907799E0C3940850F3
:100096000302087C9077A6E0FF9077DFE06F6003AD
:1000A60002087C9077A7E0FF9077E0E06F6003029C
:1000B600087C9077A8E0FF9077E1E06F6003020884
:1000C6007C9077A9E0FF9077E2E06F600302087CFE
:1000D6009077AAE0FF9077E3E06F600302087C90D8
:1000E60077ABE0FF9077E4E06F600302087C9077DF
:1000F600DEE0B44415907715E0B4FF0E63A20190DC
:1001060080A863A2017F06122B09907AF2E06003B1
:100116007401F0907AF37464F09077DE7452F09084
:1001260077DDE0646D60030202A37BFF7A13796ECC
:100136001218F97BFF7A1379889077A6E0F52FA33A
:10014600E0F530A3E0F531A3E0F532A3E0F533A303
:10015600E0F5341218F9752FFF7530137531E57512
:1001660032FF7533137534F17BFF7A1379BE12189B
:10017600F97BFF7A1379FA1218F97BFF7A14796002
:100186001218F97BFF7A14798D9077ACE0F52FA3DE
:10019600E0F530A3E0F531A3E0F5321218F97BFF64
:1001A6007A1479B79077B5E0F52FA3E0F530A3E0A0
:1001B600F531A3E0F5321218F97BFF7A1479E59050
:1001C60077B9E0F52FA3E0F530A3E0F531A3E0F52C
:1001D600321218F97BFF7A1579139077A2E0F52F82
:1001E600A3E0F530A3E0F531A3E0F5321218F97B70
:1001F600FF7A15793690779EE0F52FA3E0F530A3C8
:10020600E0F531A3E0F5321218F97BFF7A15795340
:100216009077BDE0F52F1218F97BFF7A15797D12DC
:1002260018F97BFF7A1579A6A20EE433F52F12187A
:10023600F97BFF7A1579D6907AE8E0F52F1218F94E
:100246007BFF7A167901907AF2E0F52F1218F97B86
:10025600FF7A16793490771BE0F52F1218F97BFF99
:100266007A167962A201E433F52F1218F97BFF7A28
:1002760016798E907AE2E0F52FA3E0F530A3E0F54B
:1002860031A3E0F532A3E0F533A3E0F5341218F913
:10029600123C7A7BFF7A1679D91218F9229077DD0B
:1002A600E0644C70527E167FDF1237579077E5E098
:1002B600F527A3E0F528E4F5297D03AF28AE27123C
:1002C60039F67E177F1A123757AE27AF28E4FB7D23
:1002D60010123BA67E177F1D12375774102528F57E
:1002E60028E43527F5270529E529C3941040CA7E59
:1002F600177F1D123757229077DDE0646C705CF52E
:100306002B7E177F1F123757E4F52AAF2B7E007D11
:10031600031239F67E177F1A123757E4F529A82BF0
:10032600E6FF74E72529F582E43477F583EFF005D7
:100336002B0529E529B410E67E777FE7E4FB7D10DF
:10034600123BA67E177F1D123757052AE52AC3944E
:100356000840B87E177F1D123757229077DDE0647C
:100366004B7061F52974CF2529F582E43477F5833E
:10037600E0603274CF2529F582E43477F583E0F422
:10038600602374CF2529F582E43477F583E0FF7482
:10039600E52529F582E43477F583E0B507100529CC
:1003A600E529B408C09075697432F0020873907735
:1003B600DD7421F0300A030208737E177F5A123764
:1003C600570208739077DDE0B4521A200A077E17A9
:1003D6007F621237579077DD7472F07E777FDD7D0E
:1003E60008124306229077DDE064497045200A072B
:1003F6007E177F6D1237579077E5E0F527A3E0F576
:1004060028E4F529852882852783E0FF74E72529D6
:10041600F582E43477F583EFF00528E528700205C8
:10042600270529E529B480DC7E777FDD7D8A1243A6
:1004360006229077DDE064437079A3E0645270464B
:10044600200A077E177F751237579077E5E0F52764
:10045600A3E0F528E4F529852882852783E493FF20
:1004660074E72529F582E43477F583EFF00528E56E
:1004760028700205270529E529B480DB7E777FDD14
:100486007D8A124306229077DEE0645760030208F5
:100496007C9077E5E0F527A3E0F52874E72529F5B4
:1004A60082E43477AD82FC7B80AF28AE27124836D3
:1004B6000208739077DDE06444600302054A907792
:1004C600E5E0FF64447003020873EFB4310CC20A1E
:1004D6007E177F7E1237570208739077E5E0B430B7
:1004E6000CD20A7E177F8A1237570208739077E577
:1004F600E0B4320CD20B7E177F971237570208737F
:100506009077E5E0B4330CC20B7E177FA512375700
:100516000208739077E5E0B4340CD20C7E177FB4F2
:100526001237570208739077E5E0B4350CC20C7E9B
:10053600177FC11237570208739077E5E0FF120064
:100546001E020873907569E07013200A077E177FF4
:10055600CF1237579077DD7421F0020873907569D2
:100566007432F09077DDE0FFB4510A908000748019
:10057600F0C2AF80FEEF64577045200A077E177FF2
:10058600DD1237579077E6E0907799F0E4F52990F9
:100596007799E0FFE529C39F400302087374E725B6
:1005A60029F582E43477F583E0FF9077E5E02529A5
:1005B6002414F582E43476F583EFF0052980D09093
:1005C60077DDE064536003020678200A077E177F12
:1005D600E81237579077A6E0FF90761DE06F703CE3
:1005E6009077A7E0FF90761EE06F70309077A8E0D6
:1005F600FF90761FE0B507249077A9E0FF9076205C
:10060600E0B507189077AAE0FF907621E0B5070CD1
:100616009077ABE0FF907622E06F60169077DD74FE
:1006260021F0300A030208737E177FF7123757024C
:100636000873E4F529E4F50D74142529F582E434EC
:1006460076F583E0FDAF291248F70529E529C3941D
:10065600FE40E29080007480F0C2AFE4907FF0F03C
:10066600A3F0907FFD74AAF0A374FFF0A37455F075
:1006760080FE9077DDE0644F704C9077E5E0F527DB
:10068600A3E0F528E5284527700A200A077E187F8B
:1006960000123757200A077E187F07123757E4F5EE
:1006A6002974E72529F582E43477F583E0852882E5
:1006B600852783F00528E528700205270529E52901
:1006C600B480DE0208739077DDE0FFB445279080A2
:1006D600007480F09077E5E0FDA3E0907FF0CDF028
:1006E600A3EDF0C2AF907FFD74AAF0A374FFF0A350
:1006F6007455F080FEEF646560030208739077E539
:10070600E0FFA3E0907FF0CFF0A3EFF0E4F527F54C
:1007160028D3907FF1E09528907FF0E0952740213F
:10072600E4F50D2528FFE5273478FE7B80AD28AC5F
:100736002712483674802528F528E43527F52780C2
:10074600D07E187F09124178EF4E60201200039088
:1007560077ACEFF01200039077ADEFF01200039044
:1007660077AEEFF01200039077AFEFF07E187F0FB1
:10077600124178EF4E60201200039077B5EFF01229
:1007860000039077B6EFF01200039077B7EFF01200
:1007960000039077B8EFF07E187F15124178EF4E80
:1007A60060201200039077B9EFF01200039077BA39
:1007B600EFF01200039077BBEFF01200039077BCC6
:1007C600EFF07E187F1B124178EF4E602012000377
:1007D6009077A2EFF01200039077A3EFF0120003D8
:1007E6009077A4EFF01200039077A5EFF07E187FC4
:1007F60021124178EF4E602012000390779EEFF0B1
:1008060012000390779FEFF01200039077A0EFF0AD
:100816001200039077A1EFF07E187F27124178EF40
:100826004E60081245D89077BDEFF0E4F529E4F55F
:100836000DE52904FF749E2529F582E43477F583B6
:10084600E0FD1248F70529E529C3944340E090806E
:10085600007480F0C2AFE4907FF0F0A3F0907FFDCB
:1008660074AAF0A374FFF0A37455F080FE7E777F20
:06087600DD7D08124306BF
:01087C002259
:1047FE00AE07EEC39430400BEED394395005EE2441
:10480E00D0FF22EEC39461400BEED394665005EEBA
:10481E0024A9FF22EEC39441400BEED394465005DB
:08482E00EE24C9FF22AF0622AF
:104A8D00907714E004F07006907713E004F09077BF
:0A4A9D0013E0FEA3E0FF1247BC2265
:10000300124A8D1247FEEFC454F0FEC006124A8D09
:080013001247FED0E02FFF228E
:1045D800E4907C30F0124A8D907C31EFF0C3943037
:1045E8004018E0FFD394395011907C30E0246CF5EA
:1045F80082E43475F583EFF08011907C30E0246C10
:10460800F582E43475F583E4F0800C907C30E004A6
:10461800F0E0D3940840BE752F0075300075310066
:0C462800E4F5327B017A75796C122BE00E
:014634002263
:044178008E2C8F2DCD
:10417C00907713E4F0A374FFF0124A8DEF606EF4A5
:10418C00606B852D82852C83E493B507EC752E012D
:10419C00E52D252EF582E4352CF583E493602590EE
:1041AC007714E0252EFF907713E03400FE1247BC05
:1041BC00E52D252EF582E4352CF583E493B5070423
:1041CC00052E80CCE52D252EF582E4352CF583E4E7
:1041DC009370A6E52E24FFFFE434FFFE907714E0E5
:1041EC002FF0907713E03EF07E007F0122E4FEFF7B
:0141FC0022A0
:103671007E187F58124178EF4E70037F01227E1829
:103681007F5B124178EF4E600C124A8DEF24D024FB
:10369100FF920E8002D20E7E187F61124178EF4EAA
:1036A100600C124A8DEF24D0907AE8F08005E49006
:1036B1007AE8F07E187F67124178EF4E600C124A6B
:1036C1008DEF24D0907AF2F08005E4907AF2F07ECA
:1036D100187F6D124178EF4E600C124A8DEF24D0A5
:1036E10090771BF08005E490771BF07E187F7312B2
:1036F1004178EF4E600C124A8DEF24D024FF9201E5
:103701008002C2019077A663A201907AE263A201CE
:103711007F06122B0930013B7E187F79124178EF29
:103721004E6030120003907AE2EFF0120003907ABB
:10373100E3EFF0120003907AE4EFF0120003907AC5
:10374100E5EFF0120003907AE6EFF0120003907AB1
:06375100E7EFF07F00220B
:10266400C201E4907AF2F0D20EC204907AE8F090BB
:10267400771BF09077A663A201907AE263A2017FB0
:1026840006122B09E4F527E52775F003A4247FF54A
:1026940082E43418F583E493FB740193FA7402938F
:1026A400F91221CA7003022856E4F528F529FD74AD
:1026B400942DF582E43475F583E0FF70030228510C
:1026C400E52775F003A4247FF582E43418F583E448
:1026D40093FB740193FA740293F98528827583003D
:1026E4001221E3FEEFB50608752901052802284DDD
:1026F400E529700302284DEE6003022848E52724EB
:10270400FE60281470030228301470030228341465
:10271400700302283C14700302284024056003025D
:102724002851907AF27401F0022851D20174942D48
:10273400F582E43475F583E0FF642D7003022851BB
:102744001247FEEFC454F0FC74952DF582E4347501
:10275400F583E0FF1247FEEF2C907AE2F074962D99
:10276400F582E43475F583E0FF1247FEEFC454F0BC
:10277400FC74972DF582E43475F583E0FF1247FE6F
:10278400EF2C907AE3F074982DF582E43475F58398
:10279400E0FF1247FEEFC454F0FC74992DF582E477
:1027A4003475F583E0FF1247FEEF2C907AE4F07461
:1027B4009A2DF582E43475F583E0FF1247FEEFC4E9
:1027C40054F0FC749B2DF582E43475F583E0FF121C
:1027D40047FEEF2C907AE5F0749C2DF582E4347575
:1027E400F583E0FF1247FEEFC454F0FC749D2DF511
:1027F40082E43475F583E0FF1247FEEF2C907AE60D
:10280400F0749E2DF582E43475F583E0FF1247FEE3
:10281400EFC454F0FC749F2DF582E43475F583E025
:10282400FF1247FEEF2C907AE7F08021D204801D3E
:10283400907AE87401F08015C20E801190771B74B1
:1028440001F08009E4F529F5280D0226B3052702D5
:02285400268BD1
:01285600225F
:1046E9009079DEE0C3947C503D9079DEE0FE04F0E1
:1046F900741C2EF582E43477F583EFF0BF0A279016
:1047090079DEE0FF04F0741C2FF582E43477F58339
:10471900E4F09079DEE0FF1243889079DE7408F0C6
:0747290090771DE004F0226F
:104690009080007480F090779E63A201F583F5828C
:1046A00063A2017F08122B099077A663A201908074
:1046B0008863A2017F0A122B09908092E4F0A37410
:1046C00032F0A37401F09077B0E0FF9080B1F090E9
:1046D00080E1EFF09080957455F0A3F09080007425
:0946E00001F09080097470F022D1
:10448100908009E04410F09080A0E0706C9080A1D1
:104491007482F09080A874FFF0A3F0A3F0A3F07FE2
:1044A100039080AEEFF07FCBA3EFF07F039080AC61
:1044B100EFF0A374CBF09080007402F0907C221294
:1044C100231F00000000907C22E0908040F0907C4F
:1044D10023E0908041F0907C24E0908042F0907C39
:1044E10025E0908043F0A3E4F0A3F0A3F0A3F090C3
:0944F1008018F0A3F0A3F0A3F081
:0144FA00229F
:10457500908009E04440F09080D17482F09077B14A
:10458500E0FF9080DEF09077B2E0FF9080DFF09062
:1045950080027402F0907C2612231F000000009018
:1045A5007C26E0908058F0907C27E0908059F09030
:1045B5007C28E090805AF0907C29E090805BF0A305
:1045C500E4F0A3F0A3F0A3F0908030F0A3F0A3F003
:0245D500A3F051
:0145D70022C1
:1044FB00908009E04420F09080B8E0706C9080B917
:10450B007482F07F039080C6EFF07FCDA3EFF07F36
:10451B00039080C4EFF0A374CDF09080C074FFF0D3
:10452B00A3F0A3F0A3F09080017402F0907C2A1208
:10453B00231F00000000907C26E090804CF0907CC4
:10454B0027E090804DF0907C28E090804EF0907C9E
:10455B0029E090804FF0A3E4F0A3F0A3F0A3F09038
:09456B008024F0A3F0A3F0A3F0FA
:014574002224
:104282008C278D28A907EAFDE975F018A424ACFF54
:10429200E5F034808F82F583EDF0EBFDE975F018DF
:1042A200A4FFAEF024ACFBEE34808B82F583A3ED49
:1042B200F08528828C83E0FDEF24A8FFEE3480FE97
:1042C2008F82F583EDF08528828C83A3E08F828E26
:1042D20083A3F0852882852783A3A3E0FDE975F0F7
:1042E20018A424A8FFE5F03480FE8F82F583A3A3EF
:1042F200EDF08528828C83A3A3A3E08F828E83A313
:04430200A3A3F0225F
:064306008D2CAB07AA0696
:10430C00907C22E0FCA3E0FDA3E0FEA3E0F5308E60
:10431C002F8D2E8C2DAE02AF038E838F8263A20164
:10432C00E52F540744C0F58385308263A201AF2C7E
:10433C00122B72908000E020E5F9E4FCFDFEE530E4
:10434C00252CF530EE352FF52FED352EF52EEC35E1
:10435C002DF52D908040E52DF0A3E52EF0A3E52F53
:10436C00F0A3E530F09080007420F0AF30AE2FADAC
:0B437C002EAC2D907C22122313AF2CDE
:014387002213
:064406008D27AB07AA069A
:10440C00907C26E0FCA3E0FDA3E0FEA3E0F52B8E60
:10441C002A8D298C28AE02AF038E838F8263A20172
:10442C00E52A540744D0F583852B8263A201AF277C
:10443C00122B72E4FCFDFEE52B2527F52BEE352A1D
:10444C00F52AED3529F529EC3528F528908058E525
:10445C0028F0A3E529F0A3E52AF0A3E52BF0908042
:10446C00027420F0AF2BAE2AAD29AC28907C26121A
:04447C002313AF2730
:014480002219
:023D4E008F28BC
:103D5000908001E030E5037F0022907C2AE0FCA304
:103D6000E0FDA3E0FEA3E0F52C8E2B8D2A8C29909C
:103D70007AE263A201E52B540744C8F583852C82BF
:103D800063A2017F06122B88E52C2406F52CE4356E
:103D90002BF52BE4352AF52AE43529F5299079E02D
:103DA00063A201E52B540744C8F583852C8263A2E6
:103DB00001AF28122B88E4FCFDFEE52C2528F52C0C
:103DC000EE352BF52BED352AF52AEC3529F5299022
:103DD000804CE529F0A3E52AF0A3E52BF0A3E52C20
:103DE000F09080017420F0AF2CAE2BAD2AAC29905E
:073DF0007C2A122313AF2807
:013DF70022A9
:10356D009081E0E0F5270527052705270527052785
:10357D0005270527052705270527908010E0F52A43
:10358D00A3E0F52BA3E0F52CA3E0F52D9081E1E070
:10359D00F5270527052705270527052705270527CE
:1035AD00052705270527908014E0F52EA3E0F52FBC
:1035BD00A3E0F530A3E0F531E530B52C08E531B5E4
:1035CD002D037F0022E4F527E530540744E0F58311
:1035DD0085318263A2019077DD63A2017F08122BF2
:1035ED00A09077DF63A20190771563A2017F061289
:1035FD002B099077DDE0F528A3E0F529E4F5279078
:10360D0077DDE0702AA3E024F8F527E53054074470
:10361D00E0F58385318274082582F582E43583F5E2
:10362D008363A2019077DD63A201AF27122BA0AEB9
:10363D0028E4FCFDE5312529F531E5303EF530ED89
:10364D00352FF52FEC352EF52E908014E52EF0A3A9
:10365D00E52FF0A3E530F0A3E531F0908000744044
:03366D00F0AF2794
:013670002237
:102F22009081E6E0F52705270527052705270527D0
:102F320005270527052705270527908028E0F52A7C
:102F4200A3E0F52BA3E0F52CA3E0F52D9081E7E0BB
:102F5200F52705270527052705270527052705271F
:102F620005270527052790802CE0F52EA3E0F52FF5
:102F7200A3E0F530A3E0F531E4F527E530B52C0AFE
:102F8200E531B52D05C20802307CE530540744F026
:102F9200F58385318263A2019077DD63A2017F0808
:102FA200122BA09077DDE0F528A3E0F529E529456D
:102FB2002870099080027410F07F0022907AE9E074
:102FC200FFF4602D9077DFE06F7076907AEAE0FF91
:102FD2009077E0E06F706A907AEBE0FF9077E1E043
:102FE2006F705E907AECE0FF9077E2E06F60228093
:102FF200509077DFE0907AE9F09077E0E0907AEA1B
:10300200F09077E1E0907AEBF09077E2E0907AEC62
:10301200F09077DDE0702AA3E024F8F527E530543C
:103022000744F0F58385318274082582F582E43500
:1030320083F58363A2019077DD63A201AF27122B90
:10304200A0AE28E4FCFDE5312529F531E5303EF559
:1030520030ED352FF52FEC352EF52EAF2DAE2CADF4
:103062002BAC2AAB31AA30A92FA82ED312230240AF
:10307200099080027410F07F002290802CE52EF0DF
:10308200A3E52FF0A3E530F0A3E531F090800274C0
:0430920040F0AF2734
:013096002217
:103097009081E3E0F527052705270527052705275D
:1030A7000527052705270527052790801CE0F52A12
:1030B700A3E0F52BA3E0F52CA3E0F52D9081E4E048
:1030C700F5270527052705270527052705270527A9
:1030D700052705270527908020E0F52EA3E0F52F8B
:1030E700A3E0F530A3E0F531E4F527E530B52C0A88
:1030F700E531B52D05C2090231E2E530540744E850
:10310700F58385318263A20190746963A2017F0E02
:10311700122BB6907469E0F528A3E0F52990747135
:10312700E0FFF46045907AE2E0FEEF6E706EA3E098
:10313700FF907472E06F7064907AE4E0FF907473AC
:10314700E06F7058907AE5E0FF907474E06F704C10
:10315700907AE6E0FF907475E06F7040907AE7E050
:10316700FF907476E06F60048032D2D9907469E082
:10317700702AA3E024F2F527E530540744E8F583E5
:10318700853182740E2582F582E43583F58363A247
:103197000190746963A201AF27122BB6AE28E4FC35
:1031A700FDE5312529F531E5303EF530ED352FF5D3
:1031B7002FEC352EF52EAF2DAE2CAD2BAC2AAB3127
:1031C700AA30A92FA82ED31223025006E529452895
:1031D70070099080017410F07F0022908020E52E06
:1031E700F0A3E52FF0A3E530F0A3E531F0908001DF
:0531F7007440F0AF2759
:0131FC0022B0
:043757008E2C8F2DF8
:10375B00907C22E0FCA3E0FDA3E0FEA3E0F5338E1A
:10376B00328D318C30E533FFE5325407FEE42FF513
:10377B002FEE34C0F52E852F82F5837423F0052FA1
:10378B00E52F7002052E532EC7F582852E83740A02
:10379B00F0052FE52F7002052E532EC79077A663E9
:1037AB00A201852E83852F8263A2017F06122B72C5
:1037BB007406252FF52FE4352EF52E852C83852DBC
:1037CB008263A201852E83852F8263A201122B5661
:1037DB00908000E020E5F9E4FCFDFE907C22E0F80F
:1037EB00A3E0F9A3E0FAA3E02FFFEE3AFEED39FDDB
:1037FB00EC38FCEF2408FFE43EFEE43DFDE43CFC2A
:10380B00907C22122313907C22E0908040F0907CDD
:10381B0023E0908041F0907C24E0908042F0907CFB
:0C382B0025E0908043F09080007420F0B5
:01383700226E
:063BA6008E2C8F2D8D2EE8
:103BAC00907C22E0FCA3E0FDA3E0FEA3E0F5348EC4
:103BBC00338D328C31E534FFE5335407FEE42FF5B9
:103BCC0030EE34C0F52F853082F5837423F0053048
:103BDC00E5307002052F532FC7F582852F83EBF04C
:103BEC000530E5307002052F532FC79077A663A2DE
:103BFC0001852F8385308263A2017F06122B72749C
:103C0C00062530F530E4352FF52F852C83852D8254
:103C1C0063A201852F8385308263A201AF2E122B04
:103C2C0072908000E020E5F97408252EF52EFFE453
:103C3C00FCFDFEE5342FF534EE3533F533ED35323E
:103C4C00F532EC3531F531908040E531F0A3E532B9
:103C5C00F0A3E533F0A3E534F09080007420F0AFCE
:0D3C6C0034AE33AD32AC31907C2212231304
:013C79002228
:024388008F4064
:10438A00907C22E0FCA3E0FDA3E0FEA3E0F5448ECE
:10439A00438D428C41E544FFE5435407FEE42FFF79
:1043AA00EE34C090771C63A201F5838F8263A20169
:1043BA00AF40122B72908000E020E5F9E4FCFDFE8C
:1043CA00E5442540F544EE3543F543ED3542F542E3
:1043DA00EC3541F541908040E541F0A3E542F0A378
:1043EA00E543F0A3E544F09080007420F0AF44AEBA
:0B43FA0043AD42AC41907C2212231323
:014405002294
:0639F6008E2C8F2DAB05A5
:1039FC00907C22E0FCA3E0FDA3E0FEA3E0F5338E77
:103A0C00328D318C30E533FFE5325407FEE42FF56F
:103A1C002FEE34C0F52E852F82F5837423F0052FFD
:103A2C00E52F7002052E532EC7F582852E83EBF001
:103A3C00052FE52F7002052E9077A663A201852E27
:103A4C0083852F8263A2017F06122B727406252FA9
:103A5C00F52FE4352EF52E532EC7E52C852F8285B8
:103A6C002E83F0052FE52F7002052E532EC7F582FD
:103A7C00852E83E52DF0052FE52F7002052E532E94
:103A8C00C7908000E020E5F9E533240AF533E435EE
:103A9C0032F532E43531F531E43530F53090804093
:103AAC00E530F0A3E531F0A3E532F0A3E533F09077
:103ABC0080007420F0AF33AE32AD31AC30907C224C
:033ACC00122313AF
:013ACF0022D4
:103E9400E4F527E5272401FFE433FE1247BC749EB2
:103EA4002527F582E43477F583EFF00527E527C36A
:103EB400943F40DFE4F527E527247FFFE433FE1237
:103EC40047BC74942527F582E43475F583EFF074C8
:103ED400942527F582E43475F583E0FF6003B4FF8D
:103EE4001D74942527F582E43475F5837420F074E9
:103EF400952527F582E43475F583E4F080090527D8
:103F0400E527C3948040B0E4907613F0F527AF27FB
:103F14007E001247BC74142527F582E43476F583B9
:0B3F2400EFF00527E527C394FE40E303
:013F2F00226F
:104A5000E4FDFCC3ED9FEC9E5015E4FBFA0BBB009C
:0F4A6000010ABA01F8BB90F50DBD00010C80E40E
:014A6F002224
:0D4AF0004390014390025390FE5390FD222D
:0D4AFD005390FD5390FE4390024390012220
:0E4AD2005390FD439002E5905408FF5390FD71
:014AE00022B3
:0D4B0A005390FD4390014390025390FD2213
:074B3300AE071FEE70FA222D
:0248CB00AD0737
:1048CD00E4FC5390FDEDA804088002C333D8FC30FE
:1048DD00E70543900180035390FE7F05124B334350
:0948ED0090020CBC08DC5390FDA4
:0148F600229F
:10494B00E4FF5390FD7E07439002E59030E00D7439
:10495B0001A806088002C333D8FC42075390FD1E02
:08496B00C3EE6480948050DF6C
:014973002221
:1048F700AB05AA07124AF07FA01248CB124AD2AFE3
:10490700021248CB124AD2AF031248CB124AD21234
:0A4917004AFD7F0A7E00124A50227A
:0447BC00AB07AA0697
:1047C000C3EB94FFEA9400400DE42BF58274773A32
:1047D000F583E493FF22124AF07FA01248CB124ADD
:1047E000D2AF031248CB124AD2124AF07FA112482C
:0D47F000CB124AD212494B124B0A124AFD5D
:0147FD002299
:024836008B2CC9
:10483800A2AF921DC2AF85A22D53A2FE8E838F8296
:1048480005A28C838D827409122BCEE52C53A2FE0F
:1048580043A220122BD053A2DF852DA2A21D92AF16
:01486800FF50
:01486900222C
:104A7000A2AF921DC2AF8C838D82EF122BCE43A2C8
:0C4A800020122BD053A2DFA21D92AFFF2A
:014A8C002207
:0249C3008F273C
:1049C500A2AF921DC2AFE4F5838D827406122BCE81
:1049D500E52743A220122BD053A2DFA21D92AF7F61
:0149E50001D0
:0149E60022AE
:0249E7008F2718
:1049E900A2AF921DC2AFE4F5838D82740A122BCE59
:1049F900E52743A220122BD053A2DFA21D92AF7F3D
:014A090001AB
:014A0A002289
:102A2E00A907E7FFA805EF93C3966008403B74FC27
:102A3E002FFF80F00F08EF93C3966008402B74FBB6
:102A4E002FFF80E00F08EF93C3966008401B74FAC7
:102A5E002FFF80D00F08EF93D3966008400B74F9C8
:102A6E002FFF80C01F1F1F1F1FEF54FEF80303F719
:102A7E00E893FC08E893FD08E893FE08E893FF222C
:102A8E0009E993C39D6008402974FB29F980F10977
:102A9E00E993C39E6008401A74FA29F980E209E9A5
:102AAE0093D39F6008400B74F929F980D319191933
:102ABE001919E9C313C313FF22740093F8ECC398DA
:102ACE004024701F740193F8EDC39840197014746C
:0E2ADE000293F8EEC398400E7009740393F84B
:102AEC00EFC39840037F00227F0122EDF8E6F00847
:102AFC00A3DFFA22EDF8E0F608A3DFFA22E0A363E5
:102B0C00A201F0A363A201DFF475A20022E0A3638B
:102B1C00A201F0A363A201E0A363A201F0A363A24C
:102B2C0001E463A201F0A363A201DFE175A200221C
:102B3C00E0A363A2016DFE936CFDEE058393FC157F
:102B4C008363A201DFEA75A200227F00E493A363F2
:102B5C00A201F00F600CA3E583C2E3F58363A2012D
:102B6C0080EA75A20022E0A363A201F0A3E583C270
:102B7C00E3F58363A201DFEE75A20022E0A363A25A
:102B8C0001F0A3E583C2E4D2E3F58363A201DFEC99
:102B9C0075A20022E583C2E3F583E0A363A201F0F2
:102BAC00A363A201DFEE75A20022E583C2E4D2E3A7
:102BBC00F583E0A363A201F0A363A201DFEC75A28D
:102BCC000022F922C002C004C00612FFF0D006D0C9
:042BDC0004D00222FD
:10405E000A536572763A004572724C656E210A00FB
:10406E00205544502054696D654750530A00200A6C
:10407E00444154414752414D3A20002043414E2085
:10408E0054696D654750530A00205472617373531F
:10409E00656E644552520A000ACEF8C4EBE8EDFB99
:1040AE0043414E210A000A45727241647243414EE9
:1040BE003A000A00205265496E69742043414E0A47
:1040CE00002043414E283029203E20544F210A0023
:0E40DE0020545520300A0020545520310A008D
:03001E00E4FF22DA
:10497400C2A9438902758C48758A4875D90475DBC8
:104984004875DC4875DD4875DE48E4F5E9F5F9D28B
:08499400D9C2DAD28CD2DE2276
:10489D00C2D9907B08E07013E5E92419F5EB30D708
:1048AD0006E5F904F5FB2285F9FB22E5E924C8F5B7
:0E48BD00EB30D706E5F904F5FB2285F9FB2266
:10473000C2D9907B08E0702C302A16E5E92432F5C6
:10474000EB30D707E5F904F5FB800385F9FBC22AB6
:1047500022E5E92405F5EB30D706E5F904F5FB225F
:1047600085F9FB22E5E92432F5EB30D706E5F904BB
:07477000F5FB2285F9FB2295
:10499C00124974907B08E0C394645006123AD0120A
:1049AC00489D120022D229E4F556907C20F0F54562
:0749BC00F55AC22AF558224A
:10477700EF24FCF545200A127E407F5E1237577EF4
:10478700777FE1E4FBAD45123BA6E545D3940D40A9
:1047970010200A077E407F65123757E4F545D22778
:1047A700229077E163A201907C1063A201AF4512CA
:0547B7002B09C22722BE
:0F4AE100D3EF6480948D5006E55A70028F5A22ED
:101EED0020D903021FCA202903021FCAE55A6052D6
:101EFD00907469540FFF7D47122B00E54764017004
:101F0D001E907471E0B4FF0ED22B200A127E407F1A
:101F1D006E1237578009302B06E4F55A021FCA128C
:101F2D00489D123838200A077E407F7C1237572093
:101F3D000A0B7E747F69E4FBAD5A123BA6E4F55A99
:101F4D00807BE5456043907C14E02405F527D39410
:101F5D000D4007E4F545D2278063907C10E52754AA
:101F6D000FFF7D47122B00E54730E702D22AE547E8
:101F7D00B40109302B06E54A6401600312383812AA
:101F8D00489DE4F545D2278034E557601E907AF4DC
:101F9D00540FFF7D47122B00E547B40103202B039F
:101FAD0012383812489DE4F5578012200F0C907BA3
:101FBD0008E0C3946450031241FD12489D123F3056
:101FCD008F27EF700302209B124730E4F558E54749
:101FDD00547EB54703124635E547B4010CD22B208C
:101FED000A077E407F89123757E559C394C8502D93
:101FFD0030032AE547B4420DE54AB4020890771B39
:10200D00E06401601874092559F582E4347BF58389
:10201D00E5272559F5597D47AF27122AF7300121BC
:10202D00E54720E71C9079E07D47AF27122AF7AFEF
:10203D0027123D4EEF700A200A077E407F97123718
:10204D0057E54754817047E527D3940D400C200A7E
:10205D003D7E407FA61237578034E549D394074023
:10206D0028200A2A7E407FB412375790756C7D4721
:10207D00AF27122AF77E757F6CE4FBAD27123BA6C6
:10208D007E407FC01237578005AF271231FD300DCE
:10209D002030001B907B08E0C3946450120558E576
:1020AD005894F0400A9080007480F0C2AF80FEC258
:1020BD000D2002030221C4906001E004F07006902F
:1020CD006000E004F0E5566031D3940140041556EC
:1020DD008028907C20E004F0E0D39403400D200A8A
:1020ED00077E407FC212375712499C200A077E4057
:1020FD007FCF123757E4F556D229302843E5577074
:10210D003F907AF404F0A37408F0A37480F0A374E4
:10211D0001F0A37406F0907C0BE0907AF9F0907CBE
:10212D000CE0907AFAF0907C0DE0907AFBF0907CC8
:10213D000EE0907AFCF0E4A3F0A3F075570BC228E3
:10214D00302672907C09E07035E5577031907AF445
:10215D007442F0A37408F0907C0AE0907AF6F09047
:10216D007C0FE0907AF7F0A37401F0755706200A02
:10217D00077E407FDE123757907C09E004F0907C9B
:10218D0009E06402702FE557702B907AF47402F019
:10219D00A37408F0907C0AE0907AF6F0A3F0A37493
:1021AD0001F0755706200A077E407FE512375790DC
:0C21BD007C09E004F0C202122D84C20074
:0121C90022F3
:10486A00E559602CE49078DDF0A3E559F0907AE1FF
:10487A00E09078DFF0A37419F0907B0963A20190AD
:10488A0078E163A201AF59122B09E4F5597F01229D
:03489A007F00227A
:0B4B1700302705C2277F01227F00220B
:0100210022BC
:064B4100E4F559F54522E0
:0A4B2200E490756CF0A3F0A3F022FC
:074B3A0020457272210A0000
:104AA700EF600A7B10E4FD7F0C124921227B107D09
:074AB700107F0C12492122BF
:103AD000D29475C353C29475C5C0E5C4B480FB8548
:103AE000C528D2947DE07F0F124A2F907B08E044D6
:103AF00080FD7F2A124A2F7D247F29124A2F7D04C0
:103B00007F28124A2FE4FD7F2B124A2F752A20E4CA
:103B1000F529E4FDAF2A124A2F052A0529E529C314
:103B2000940840EEE4F52AF529E4FDAF2A124A2F65
:103B3000052A0529E529C3940C40EE7D087F05126E
:103B40004A2F752A10E4F529E4FDAF2A124A2F0501
:103B50002A0529E529C3940C40EE7D3C7F0C124ACE
:103B60002F7D077F0F124A2F7DFF7F2B124A2F7563
:103B70002A30E4F528E4F529E4FDAF2A124A2F059E
:103B80002A0529E529C3940E40EE052A052A0528B1
:103B9000E528C3940340DE7D047F60124A2FE4FDD4
:053BA0007F70124A2FA6
:013BA50022FD
:104A0B00C29475C503E5C4B480FBAEC58FC5E5C4C0
:104A1B00B480FBAEC5E4F5C5E5C4B480FBAEC5D22E
:034A2B0094AF063F
:014A2E002265
:104A2F00C29475C502E5C4B480FBAEC58FC5E5C49D
:104A3F00B480FBAEC58DC5E5C4B480FBAEC5D294C2
:014A4F002244
:10492100C29475C505E5C4B480FBAEC58FC5E5C4A9
:10493100B480FBAEC58BC5E5C4B480FBAEC58DC5E7
:09494100E5C4B480FBAEC5D294BC
:01494A00224A
:10391800C29475C503E5C4B480FBAEC5EF60047EF0
:103928007080027E608EC5E5C4B480FBAEC5E4F548
:10393800C5E5C4B480FB85C546E4F5C5E5C4B480D7
:10394800FB85C547E4F5C5E5C4B480FB85C548E4F7
:10395800F5C5E5C4B480FB85C549E4F5C5E5C4B43F
:1039680080FB85C54AE4F5C5E5C4B480FB85C54B35
:10397800E54B540FFE60741EE4F5C5E5C4B480FB46
:1039880085C54CEE60651EE4F5C5E5C4B480FB85CD
:10399800C54DEE60561EE4F5C5E5C4B480FB85C58B
:1039A8004EEE60471EE4F5C5E5C4B480FB85C54FFF
:1039B800EE60381EE4F5C5E5C4B480FB85C550EE5D
:1039C80060291EE4F5C5E5C4B480FB85C551EE60E9
:1039D8001A1EE4F5C5E5C4B480FB85C552EE600B3C
:0D39E800E4F5C5E5C4B480FB85C553D29459
:0139F50022AF
:10383800907B08E0C394644003023915C29475C5AF
:1038480002E5C4B480FBAFC575C531E5C4B480FBDF
:10385800AFC5E54B540FFE8547C5E5C4B480FBAF43
:10386800C58548C5E5C4B480FBAFC58549C5E5C471
:10387800B480FBAFC5854AC5E5C4B480FBAFC58538
:103888004BC5E5C4B480FBAFC5EE606C1E854CC566
:10389800E5C4B480FBAFC5EE605E1E854DC5E5C4CA
:1038A800B480FBAFC5EE60501E854EC5E5C4B4803C
:1038B800FBAFC5EE60421E854FC5E5C4B480FBAFC3
:1038C800C5EE60341E8550C5E5C4B480FBAFC5EEB7
:1038D80060261E8551C5E5C4B480FBAFC5EE6018EF
:1038E8001E8552C5E5C4B480FBAFC5EE600A85539A
:1038F800C5E5C4B480FBAFC5D2947F02C29475C538
:0F39080081E5C4B480FBAFC5D29475560AC229BD
:01391700228D
:10463500C29475C502E5C4B480FBAFC575C541E537
:10464500C4B480FBAFC58547C5E5C4B480FBAFC521
:104655008548C5E5C4B480FBAFC58549C5E5C4B487
:1046650080FBAFC5854AC5E5C4B480FBAFC5E4F59D
:10467500C5E5C4B480FBAFC5D2947F02C29475C5AD
:0A46850082E5C4B480FBAFC5D294F7
:01468F002208
:1041FD00C29475C502E5C4B480FBAFC575C551E564
:10420D00C4B480FBAFC57472250FF582E43461F53B
:10421D0083E0F5C5E5C4B480FBAFC575C508E5C43D
:10422D00B480FBAFC57473250FF582E43461F5835B
:10423D00E0F5C5E5C4B480FBAFC575C50FE5C4B4E5
:10424D0080FBAFC5050F050F7472250FF582E434A1
:10425D0061F583E07002F50FE4F5C5E5C4B480FBAC
:10426D00AFC5D2947F02C29475C584E5C4B480FBFA
:04427D00AFC5D29463
:01428100221A
:103F30003092037F00227F2C124A0B8F28E5283015
:103F4000E209D229E4F556907C20F0E52830E558C6
:103F5000200A077E4B7F3A1237577F2D124A0B8F6C
:103F600029200A11E528FE7C00E42529FFEC3EFE0D
:103F70007D031239F6E4FBAD297F2D124921200A79
:103F80001BE52830E016E4FF123918E547FE7C00F7
:103F9000E4254BFFEC3EFE7D031239F6AB28E4FD31
:103FA0007F2C1249217F0022E4F529E52830E00D1D
:103FB000E4FF123918E54B54072405F529AB28E432
:083FC000FD7F2C124921AF29FD
:013FC80022D6
:100DF6005452414E5A004D415842005254530044F9
:100E0600454C4159004E4F4B5654004B5000424FF3
:100E16004F540043414E004E4557504B54004154E9
:100E2600004443440043414E4D4F4E0054454C3A16
:100E3600004C434C004454420054524300003E2AA6
:100E46002C312CCFE0F0E0ECE5F2F0FB20F3EFF0F4
:100E5600E0E2EBFFFEF9E5E3EE20EAEEEDF2F0EE7E
:100E6600EBEBE5F0E020CACF20C8F1E5F2FC0A0082
:100E76003E4C2C6B30312C25732C43EAEEF0EEF110
:100E8600F2FC20EDE020F8E8EDE52043414E2C3061
:100E9600202D20353030EAE1283530EC292C312060
:100EA6002D203530EAE128353030EC290A00302093
:100EB6002D20353030EAE1283530EC290031202D5F
:100EC600203530EAE128353030EC29003E532C6BD2
:100ED60030322C2562752CCCE0EAF12E20E0E4F0CD
:100EE600E5F120E1EBEEEAE020D2D128302D3829D9
:100EF6000A003E532C6B30332C2562752CCCE0EA6D
:100F0600F12E20E0E4F0E5F120E1EBEEEAE020D27C
:100F1600C8D228302D38290A003E532C6B30342C89
:100F26002562752CCCE0EAF12E20E0E4F0E5F12014
:100F3600E1EBEEEAE020D2D328302D38290A003E34
:100F4600422C6330312C2562752CC2F2EEF0E8F7A4
:100F5600EDFBE920EAEEEDF2F0EEEBEBE5F020ED4D
:100F6600E020F8E8EDE50A003E2A2C312CCFE0F02F
:100F7600E0ECE5F2F0FB20EFF0EEF2EEEAEEEBE06D
:100F860020C8F1E5F2FC20EFEE20EFEEF0F2F320C0
:100F960052533233320A003E4C2C6B30352C256CC2
:100FA600752CD1EAEEF0EEF1F2FC20EEE1ECE5ED87
:100FB600E020EDE020EFEEF0F2F32C3130302C3271
:100FC60030302C3330302C3630302C313230302C1F
:100FD600323430302C343830302C393630302C31F5
:100FE600393230302C33383430302C3537363030D7
:100FF6002C3131353230300A003E532C6B30362CD2
:101006002562752CCAEEEB2DE2EE20E1EBEEEAEE60
:10101600E220E220EFE0EAE5F2E50A003E422C6B30
:1010260030392C2562752CCDE520EFE5F0E5E4E0BE
:10103600E2E0F2FC20E4E8E0E3EDEEF1F2E8EAF3C8
:101046000A003E422C6B31302C2562752CD0E5F11E
:10105600F2E0F0F220EFF0E820EEF2F1F3F2F1F236
:10106600E2E8E820EFE5F0E5E4E0F7E820EFE0EA83
:10107600E5F2EEE2203220ECE8ED2E0A003C2100FB
:101086003C6B30313D003C6B30323D003C6B3033C5
:101096003D003C6B30343D003C6330313D003C6BE1
:1010A60030353D003C6B30363D003C6B30393D0001
:1010B6003C6B31303D0043796354530A004D6573F0
:1010C600730A00435449490A00435449540A0053D9
:1010D600705449540A0054696D655449540A000A0B
:1010E6004173796E634F55543A00CEF820E4EBE82D
:1010F600EDFB210A000A435243204552523A200092
:101106000A494E3A000A4173796E63494E3A003FE6
:101116003F3F0A000089129B24AD36BF48C15AD30F
:101126006CE57EF78108931AA52CB73EC940DB52C1
:10113600ED64FF76028B109926AF34BD4AC358D1B1
:101146006EE77CF5830A9118A72EB53CCB42D950A1
:10115600EF66FD74048D169F20A932BB4CC55ED781
:1011660068E17AF3850C971EA128B33ACD44DF5681
:10117600E960FB72068F149D22AB30B94EC75CD571
:101186006AE378F1870E951CA32AB138CF46DD5461
:10119600EB62F97008811A932CA53EB740C952DB61
:1011A60064ED76FF89009B12AD24BF36C148D35A41
:1011B600E56CF77E0A8318912EA73CB542CB50D931
:1011C60066EF74FD8B029910AF26BD34C34AD15821
:1011D600E76EF57C0C851E9728A13AB344CD56DF01
:1011E60060E972FB8D049F16A920BB32C54CD75E01
:1011F600E168F37A0E871C952AA338B146CF54DDF1
:1012060062EB70F98F069D14AB22B930C74ED55CE0
:10121600E36AF17800112332465765748C9DAFBEA0
:10122600CADBE9F810013322564775649C8DBFAEC0
:10123600DACBF9E82130021367764455ADBC8E9FB0
:10124600EBFAC8D93120120377665445BDAC9E8FA0
:10125600FBEAD8C94253617004152736CEDFEDFC90
:101266008899ABBA5243716014053726DECFFDEC80
:101276009889BBAA6372405125340617EFFECCDD70
:10128600A9B88A9B7362504135241607FFEEDCCD60
:10129600B9A89A8B8495A7B6C2D3E1F008192B3A60
:1012A6004E5F6D7C9485B7A6D2C3F1E018093B2A40
:1012B6005E4F7D6CA5B48697E3F2C0D129380A1B30
:1012C6006F7E4C5DB5A49687F3E2D0C139281A0B20
:1012D6007F6E5C4DC6D7E5F48091A3B24A5B697810
:1012E6000C1D2F3ED6C7F5E49081B3A25A4B796800
:1012F6001C0D3F2EE7F6C4D5A1B082936B7A4859F0
:101306002D3C0E1FF7E6D4C5B1A092837B6A5849DF
:101316003D2C1E0FFF0DF6FF0DFCFF0E01FF0E0507
:10132600FF0E0BFF0E11FF0E14FF0E19FF0E1DFF11
:101336000E24FF0E27FF0E2BFF0E32FF0E37FF0E79
:071346003BFF0E3FFF0E43C9
:0300230002335154
:0B335100C0E0C083C082C0D075D0185F
:10335C0030984AC298750B01AF9920100DEF64029A
:10336C00703B90616CF0D2108033301707C217534A
:10337C001F0F801ABF0904D2178022BF031085616A
:10338C006C636180536180C210750B00800F7422D6
:10339C002561F582E4346FF583EFF0056120990324
:1033AC0002345D20110302345B30166EE568B4FF05
:1033BC000B7599020568756D0002345BE568B560A4
:1033CC00137599030568906F1FE0700302345B74EA
:1033DC0001F0807BE568D395604006C211D21C8059
:1033EC006EE56D6009F5990568756D008061742254
:1033FC002568F582E43470F583E0F56D6402600BAA
:10340C00E56D64036005E56DB40905759909803FA8
:10341C00856D990568756D00803574222568F58277
:10342C00E43470F583E0FF7006C211D21C8020C218
:10343C001CEFB47C090568750832C2118011AF68A5
:10344C00056874222FF582E43470F583E0F599C297
:01345C0099D6
:09345D00D0D0D082D083D0E0323F
:103C7A007BFF7A0E79441218F9907B08E07014756C
:103C8A002FFF75300E7531B47BFF7A0E79761218D4
:103C9A00F98012752FFF75300E7531C37BFF7A0ECE
:103CAA0079761218F97BFF7A0E79D2906171E0F574
:103CBA002F1218F97BFF7A0E79F890616BE0F52FD5
:103CCA001218F97BFF7A0F791F906102E0F52F1223
:103CDA0018F97BFF7A0F7945A20FE433F52F1218F2
:103CEA00F97BFF7A0F796E1218F9907463E0FEA3DC
:103CFA00E0FFC3E49FFFE49EFEAB07FAE4F9F8FF96
:103D0A007E8C7D0AFC1222628F328E318D308C2F8E
:103D1A007BFF7A0F799D1218F97BFF7A0F79FF855D
:103D2A00692F1218F97BFF7A107922A218E433F569
:103D3A002F1218F97BFF7A107948906F1FE0F52F40
:043D4A001218F92230
:103466007E107F83124178EF4E70037F0122E49035
:103476007B08F07E107F86124178EF4E6015124A67
:103486008DBF3106907B08740AF0BF3206907B0828
:103496007464F07E107F8C124178EF4E60081245FE
:1034A600D8906171EFF07E107F92124178EF4E60F6
:1034B600081245D890616BEFF07E107F9812417824
:1034C600EF4E60081245D8906102EFF07E107F9EA5
:1034D600124178EF4E600D1245D8EC4D4E4F24FF49
:1034E600920F8002C20F7E107FA4124178EF4E60C9
:1034F600231245D8A804A905AA06AB077F007E8C2F
:103506007D0A7C001222621222F4907463EEF0A30C
:10351600EFF0800A90746374FFF0A374DCF07E1001
:103526007FAA124178EF4E60071245D88F69800353
:10353600756902E56970037569017E107FB01241F5
:1035460078EF4E600A124A8DEF24D024FF92187E3F
:10355600107FB6124178EF4E600A124A8DEF24D0E2
:06356600906F1FF07F00D2
:01356C00223C
:10285700E4F50F907C30F0907C30E075F003A42411
:102867001AF582E43413F583E493FB740193FA7445
:102877000293F91221CA7003022A2DE4907C32F0E8
:10288700A3F0907C31F0907C31E02494F582E4341D
:1028970075F583E0FF7003022A24907C30E075F021
:1028A70003A4241AF582E43413F583E493FB74013B
:1028B70093FA740293F9907C32E0F58275830012E3
:1028C70021E3FEEFB5060F907C337401F0907C3264
:1028D700E004F0022A1B907C33E07003022A1BEE0F
:1028E7006003022A12907C30E014607424FC7003A9
:1028F7000229D4147003022A021470030229A424A3
:10290700F97003022A06147003022A0A240F6003CF
:10291700022A24907C31E02494F9E43475FA7B018F
:10292700C0031B8B2F753000753100E4F532D003DF
:10293700122BE0907C34122313907C34E0F8A3E050
:10294700F9A3E0FAA3E0FB7F007E8C7D0A7C0012EE
:1029570022621222F4907463EEF0A3EFF0022A24AD
:10296700907C31E0FD2494F582E43475F583E0240E
:10297700D0906171F074952DF582E43475F583E09C
:1029870024D090616BF0907C31E02496F582E4349A
:1029970075F583E024D0906102F0022A24907C31FF
:1029A700E02494F9E43475FA7B01C0031B8B2F757F
:1029B7003000753100E4F532D003122BE0907C34FF
:1029C700122313907C37E0907B08F08050907C3185
:1029D700E02494F9E43475FA7B01C0031B8B2F754F
:1029E7003000753100E4F532D003122BE0907C34CF
:1029F700122313907C37E0F56B8022D212801ED20F
:102A070018801A906F1F7401F08012E4907C33F0E5
:102A1700907C32F0907C31E004F002288D907C307D
:062A2700E004F002285E4D
:012A2D002286
:10245D00E4906170F09061B5F0C21590616EF090EE
:10246D006F1E7405F0C211C21CC210C217E4F568CC
:10247D00F560F508F561F50B90746374FFF0A374C6
:10248D00F4F09061027402F090616BF0906171F064
:10249D00C21AD219C20F907122741EF0E4907B08FB
:1024AD00F0C212C214C213F56BC218906F1FF0D296
:1024BD0016123466EF6003122857907122E00490D3
:1024CD00616DF0E4F50F907C2E7461F0A37472F0E1
:1024DD00906171E0F50FE50FC394014007E50FD34F
:1024ED0094084003E4F50FE50F6028907C2EE47509
:1024FD00F00112221085F082F58374C4F0150F904F
:10250D007C2EE475F00112221085F082F583E50F23
:10251D00F080D490616BE0F50FE50FC39401400797
:10252D00E50FD394084003E4F50FE50F6028907C88
:10253D002EE475F00112221085F082F58374C8F037
:10254D00150F907C2EE475F00112221085F082F5A6
:10255D0083E50FF080D4906102E0F50FE50FC39491
:10256D00014007E50FD394084003E4F50FE50F6034
:10257D0028907C2EE475F00112221085F082F583EF
:10258D0074C2F0150F907C2EE475F00112221085A7
:10259D00F082F583E50FF080D4907C2EE475F00188
:1025AD0012221085F082F583E4F0907C2E75F001F7
:1025BD0012221085F082F583E4F0F50FF56A75F0BF
:1025CD0075E56AA42436F582E5F03468F583E4F008
:1025DD00E56A75F00DA42403F582E43461F583E416
:1025ED00F0F55F75F068E56AA42423F582E5F03413
:1025FD0071F58375F00DE55F122350E4F0055FE58D
:10260D005FB408DF056AE56AB408B3E4F56FF55BFE
:10261D00F55DF55EF567F56EF55FF55CF56AF566EA
:10262D00F59BC2ADF5C9D2CDD2CCC2C9C2CAF5CDCA
:10263D00F5CC907463E0F5CBA3E0F5CA85CBCD85E1
:10264D00CACCD29ED29CD2CAC2ACC298C29975B81D
:06265D001075B710D2ACAD
:012663002254
:0100220022BB
:1031FD008F2830180EE547B44209E54A6402700382
:10320D00023350E54854E324DF606D24DF6042143F
:10321D00603F24E370030232AC1470030232FE14DB
:10322D00700302332F24E2602824606003023350C0
:10323D00300B077E107FBC123757E54975F00DA492
:10324D002403F582E43461F5837D47AF28122AF714
:10325D0022300B077E107FC312375775F00DE55ED8
:10326D00A424DEF582E5F0346BF5837D47AF28129B
:10327D002AF7055E535E3F22300B077E107FC91281
:10328D00375775F00DE55BA424B6F582E5F0346192
:10329D00F5837D47AF28122AF7055B535B7F2230FC
:1032AD000B077E107FCF12375775F075E549A424B3
:1032BD0043F582E5F03468F583E54A541FFF131397
:1032CD00543F75F00D1223507D47AF28122AF77524
:1032DD00F068E549A42423F582E5F03471F583E522
:1032ED004A541FFF1313543F75F00D122350E4F091
:1032FD0022300B077E107FD512375775F068E549E0
:10330D00A42423F582E5F03471F583E54A543FFF9B
:10331D001313543F75F00D1223507D477F0D122A64
:10332D00F722300B077E107FDC12375775F075E5ED
:10333D0049A42436F582E5F03468F5837D47AF283E
:04334D00122AF72227
:103FC9008F2B90600263A20190702263A201AF2B34
:103FD900122B09E4F562F563852B6590702263A2C3
:103FE9000190111A63A201AF65AE64AD63AC6212B0
:103FF9002B3C8F658E648D638C627422252BF58230
:10400900E43470F583E563F07423252BF582E434F9
:1040190070F583E562F07422252BF582E43470F59E
:1040290083E0FFA3E0906F20CFF0A3EFF0E52B240E
:1040390002F560200A127E107FE51237577E707FE5
:1040490022E4FBAD60123BA67568FFD211C299202C
:0540590099FDD299223F
:101BF300E55E655D605875F00DE55DA424E2F58250
:101C0300E5F0346BF583E02405F52BD3940E400CFB
:101C1300200A357E107FF0123757802C75F00DE5C2
:101C23005DA424DEF582E5F0346BF58363A20174D1
:101C3300042566F582E43460F58363A201AF2B12B9
:101C43002B09E52B2566F566055D535D3F2275F08F
:101C530075E56AA42436F582E5F03468F583E0700F
:101C630003021D5AE55C705575F075E56AA4243AC4
:101C7300F582E5F03468F583E02405F52BD3940E63
:101C8300400C200A357E107FF0123757802C75F0F8
:101C930075E56AA42436F582E5F03468F58363A21A
:101CA3000174042566F582E43460F58363A201AF11
:101CB3002B122B09E52B2566F566055C2275F0755D
:101CC300E56AA42439F582E5F03468F583E0540F1E
:101CD300FFE55CD39F506575F075E56AA4243AF57A
:101CE30082E5F03468F58375F00DE55C122350E06E
:101CF3002405F52BD3940E400C200A3D7E107FF073
:101D0300123757803475F075E56AA42436F582E5F9
:101D1300F03468F58375F00DE55C12235063A2017E
:101D230074042566F582E43460F58363A201AF2B66
:101D3300122B09E52B2566F566055C22E4F55C7537
:101D4300F075E56AA42436F582E5F03468F583E49A
:101D5300F0056A536A0722056A536A07E55B656FF4
:101D6300605875F00DE56FA424BAF582E5F034618F
:101D7300F583E02405F52BD3940E400C200A357E21
:101D8300107FF0123757802C75F00DE56FA424B641
:101D9300F582E5F03461F58363A20174042566F5E9
:101DA30082E43460F58363A201AF2B122B09E52B88
:101DB3002566F566056F536F7F22E56775F00DA401
:101DC3002403F582E43461F583E06067E56775F029
:101DD3000DA42407F582E43461F583E02405F52B93
:101DE300D3940E400C200A347E107FF012375780B4
:101DF3002BE56775F00DA42403F582E43461F583C4
:101E030063A20174042566F582E43460F58363A25A
:101E130001AF2B122B09E52B2566F566E56775F0F7
:101E23000DA42403F582E43461F583E4F0056753DC
:101E3300670722056753670775F068E56EA42423D7
:101E4300F582E5F03471F58375F00DE55F122350EB
:101E5300E07003021EDB75F068E56EA42427F582AB
:101E6300E5F03471F58375F00DE55F122350E0243E
:101E730005F52BD3940E400C200A3D7E107FF01203
:101E83003757803475F068E56EA42423F582E5F0B6
:101E93003471F58375F00DE55F12235063A201746D
:101EA300042566F582E43460F58363A201AF2B1247
:101EB3002B09E52B2566F56675F068E56EA42423EA
:101EC300F582E5F03471F58375F00DE55F1223506B
:101ED300E4F0055F535F0722055FE55FC3940840A5
:091EE30008E4F55F056E536E077B
:011EEC0022D3
:102D8400300028C200906F1FE0601204F0E0D3947A
:102D9400F0400A9080007480F0C2AF80FE90616FB2
:102DA400E004F09061B5E0600214F0E508B4010CB1
:102DB400E4F508D211C2992099FDD299E50BD39478
:102DC400644007C210E4F561F50B30110F90616F98
:102DD400E0D39414400BC211D21C8005E490616FBF
:102DE400F020113EE508703A301937F528E528C37C
:102DF40095695010121BF3E5666009D394C850041A
:102E0400052880E9E566601AE4906002F0A374196D
:102E1400F0E5662402FF123FC9E4F566906000F015
:102E2400A3F0E56C7003022F21F528E4F56CF5623C
:102E3400F563E528547FF565E52854802422F5825E
:102E4400E4346FF58363A20190111A63A201AF65A4
:102E5400AE64AD63AC62122B3C8F658E648D638C63
:102E640062E52854802422F582E4346FAF82F52988
:102E74008F2A53287FE56345626022300A03022FBC
:102E8400217E107FFB123757E4FBAD28AF2AAE2911
:102E9400123BA67D03AF63AE621239F622200A2EDE
:102EA400906170E0640160147E117F06123757E46C
:102EB400FBAD28AF2AAE29123BA680127E117F0BF0
:102EC400123757E4FBAD28AF2AAE29123BA6E528FA
:102ED400B40408E490616DF0C21B22852A8285291E
:102EE40083A3E024E7702CD215E52824FCF557C30E
:102EF400940E501BE52A2402FFE43529F5838F82C2
:102F040063A201907AF463A201AF57122B0922E461
:0D2F1400F55722200A077E117F151237574E
:012F2100228D
:1040F80002087DE493A3F8E493A34003F68001F259
:1041080008DFF48029E493A3F85407240CC8C333C8
:10411800C4540F4420C8834004F456800146F6DF97
:10412800E4800B0102040810204080904B2CE47EB0
:10413800019360BCA3FF543F30E509541FFEE4938C
:10414800A360010ECF54C025E060A840B8E493A353
:10415800FAE493A3F8E493A3C8C582C8CAC583CA7E
:10416800F0A3C8C582C8CAC583CADFE9DEE780BE36
:014B32000082
:1021CA00BB010689828A83E0225002E722BBFE0213
:0921DA00E32289828A83E4932246
:1021E300BB010CE58229F582E5833AF583E02250B1
:1021F30006E92582F8E622BBFE06E92582F8E222FB
:0D220300E58229F582E5833AF583E4932214
:10221000A3F8E0C5F025F0F0E58215827002158381
:06222000E0C838F0E822DE
:1022260075F008758200EF2FFFEE33FECD33CDCC6F
:1022360033CCC58233C5829BED9AEC99E5829840F2
:102246000CF582EE9BFEED9AFDEC99FC0FD5F0D6CF
:10225600E4CEFBE4CDFAE4CCF9A88222B800C1B9F9
:102266000059BA002DEC8BF084CFCECDFCE5F0CB37
:10227600F97818EF2FFFEE33FEED33FDEC33FCEB70
:1022860033FB10D703994004EB99FB0FD8E5E4F92B
:10229600FA227818EF2FFFEE33FEED33FDEC33FC18
:1022A600C933C910D7059BE99A4007EC9BFCE99A0C
:1022B600F90FD8E0E4C9FAE4CCFB2275F010EF2F51
:1022C600FFEE33FEED33FDCC33CCC833C810D70751
:1022D6009BEC9AE899400AED9BFDEC9AFCE899F88C
:0E22E6000FD5F0DAE4CDFBE4CCFAE4C8F9221F
:0E22F400C3E49FFFE49EFEE49DFDE49CFC22FB
:10230200EB9FF5F0EA9E42F0E99D42F0E89C45F031
:0123120022A8
:0C231300ECF0A3EDF0A3EEF0A3EFF0223D
:10231F00A8828583F0D083D08212233612233612FF
:10232F002336122336E473E493A3C583C5F0C58324
:10233F00C8C582C8F0A3C583C5F0C583C8C582C808
:01234F00226B
:0C235000A42582F582E5F03583F5832298
:10189700E53B242FF8E6053B22782C302402782FED
:1018A700E475F0011223BD0221CA201DEB7F2ED261
:1018B7001D8018EF540F2490D43440D4FF30210BEF
:1018C700EF24BFB41A0050032461FFE53C60021502
:1018D7003C053FE53F7002053E30240D782CE4754A
:1018E700F0011223BDEF02235C0246E97403D22400
:1018F7008003E4C224F53B8B2C8A2D892EE4F53C2A
:10190700F53EF53FE53C60077F201218D280F5755C
:101917003DFFC21EC21DC21FC220C222C223C22552
:101927001218A0FF700D3024057F001218E3AF3F97
:10193700AE3E22B4255FC2D5C2211218A0FF24D023
:10194700B40A00501A75F00A783C30D50508B6FF7E
:101957000106C6A426F620D5047002D22080D92419
:10196700CFB41A00EF5004C2E5D221021AE3D21E07
:1019770080C6D21D80C0D21F80BCD2D580BAD222E9
:1019870080B47F201218D2201F077401B53C004095
:10199700F1121897FF1218D202190BD225D2238001
:1019A70095121897FB121897FA121897F94A4B7065
:1019B7000679B47A1B7BFF201F2EE53C602A7E0048
:1019C7008E827583001221E360060EEE653D70F08E
:1019D700C2D5EBC0E0EAC0E0E9C0E0EE121B2AD0B6
:1019E700E0F9D0E0FAD0E0FB1221CAFF60AAEBC011
:1019F700E0EAC0E0E9C0E01218D2D0E02401F9D053
:101A0700E03400FAD0E0FBE53D0460DCD53DD98049
:101A1700877BFF7A1B7926D21F809C7910800279F9
:101A270008C223C2258008D2D5790A8004790AC260
:101A3700D5E53D047002F53DE4FAFDFEFF12189767
:101A4700FC7B08201E13121897FD7B10301D0A120D
:101A57001897FE121897FF7B20EC3382D592D5504A
:101A670013C3E4301D069FFFE49EFEE4201E039D82
:101A7700FDE49CFCE4CBF8C21EEC700CCFCECDCCC1
:101A8700E824F8F870F38017C3EF33FFEE33FEED69
:101A970033FDEC33FCEB33FB994002FB0FD8E9EB4A
:101AA700301E05F8D0E0C448B21EC0E00AEC4D4E27
:101AB7004F78207B0070C2EAB53D0040BCC0E01201
:101AC7001B2CD0F0D0E0201E04C4C0E0C4B21EC05E
:101AD700F01218BBD0F0D5F0EB02190B12241C1929
:101AE700A8531A225819794C1975421A264F1A2EDB
:0F1AF700441A2E49198E431A34551A18461A18D4
:101B0600451A18471BD450197D2D19812E19A42B5F
:101B160019852319A2201BBD2A193D480000199CCE
:101B26003F3F3F00790AA2D5202014302209B91080
:101B3600020404B9080104A2D5202302500104209E
:101B46001F68921FB53C005034C0E07F203020193A
:101B56007F30A21F72237222500F121B83C21FC234
:101B660023C222C2257F30800F302203E9C0E01253
:101B760018D2302203D0E0F9D0E0B53CCC302217A1
:101B86007F30B9100C1218D27F583021077F788029
:101B960003B908031218D2301F057F2D0218D27F11
:101BA600202025F87F2B2023F322921F80CF286E3A
:101BB600756C6C2900D21E121897301EF8C21E785A
:101BC6003C30D50108F602193D2D504349581218EC
:101BD600972403B405004001E4901BCF931218C369
:0D1BE600743A1218C3D220753C04021A2272
:102BE0008B2C8A2D892EE4F538F537F536F535F539
:102BF00033F534E5304531452F6012EBC0E0EAC0D3
:102C0000E0E9C0E0AB2FAA30A9311223CDAB2C05EF
:102C10002EE52EAA2D7002052D14F91221CAF539C0
:102C2000C394094007E539D3940D40E1E5396420A8
:102C300060DBE539B42D054334038016E539B42B48
:102C400005433401800C74FF252EF52E74FF352DBD
:102C5000F52DE53260046410703FAB2CAA2DA92E2F
:102C60001221CA64306009E532702E75320A80295B
:102C70009000011221E3FF64786004EFB45813431D
:102C800034017532107402252EF52EE4352DF52D04
:102C90008007E5327003753208AB2C052EE52EAAAD
:102CA0002D7002052D14F91221CAF539C394614023
:102CB0000AE539D3947A50035339DF74D02539F5B6
:102CC00039C3940A400CE5399411406D74F92539E3
:102CD000F539E539D39532506043340185383D8567
:102CE000373C85363B85353AAF327E00E4FCFDABA0
:102CF00038AA37A936A83512236EC8ECC8C9EDC961
:102D0000CAEECACBEFCBE4FCFDFEEB2539F538EE7D
:102D10003AF537ED39F536EC38F535AF38AE37AD35
:102D200036FCAB3DAA3CA93BA83AD3122302500380
:102D3000022C99433404022C99E53420E003E4800A
:102D40002DE5304531452F601EAB2CE52E24FFF9D3
:102D5000E52D34FFFAEBC0E0EAC0E0E9C0E0AB2FBC
:102D6000AA30A9311223CDE53430E20774FFFFFE0B
:102D7000FDFC22E534AF38AE37AD36AC3530E1037B
:042D80000222F42215
:10235C00BB010689828A83F0225002F722BBFE0160
:02236C00F3225A
:10236E00E88FF0A4CC8BF0A42CFCE98EF0A42CFC0E
:10237E008AF0EDA42CFCEA8EF0A4CDA8F08BF0A48C
:10238E002DCC3825F0FDE98FF0A42CCD35F0FCEBEB
:10239E008EF0A4FEA9F0EB8FF0A4CFC5F02ECD39B0
:0F23AE00FEE43CFCEAA42DCE35F0FDE43CFC221D
:1023BD00FAE6FB0808E6F925F0F618E6CA3AF62221
:1023CD00BB011A89828A83D0F0D0E0F8D0E0F9D031
:1023DD00E0FAD0E0FBE8C0E0C0F002244B5016E973
:1023ED00F8D083D082D0E0F9D0E0FAD0E0FBC08203
:1023FD00C083022442BBFE16E9F8D083D082D0E020
:0F240D00F9D0E0FAD0E0FBC082C0830224542251
:10241C00D083D082F8E4937012740193700DA3A34F
:10242C0093F8740193F5828883E473740293686063
:06243C00EFA3A3A380DF63
:09244200EBF608EAF608E9F622BF
:09244B00EBF0A3EAF0A3E9F02292
:09245400EBF208EAF208E9F222B9
:00000001FF
